:020000020000FC
:020000000CC032
:020008005CC0DA
:1000180050C00FEF07BB08BB03E701BB0CE002BBF6
:100028000FED0DBFEE2404E6F02ED1E0DD2ECD2E2F
:10003800332400271127B801C801D8019801A80165
:1000480000936700009363000093650000936000CD
:10005800009361000093700000936C0000936D00A2
:1000680000936E0000936F0001E000936600009318
:100078006200009364000093690000936A0004E042
:100088000093680030BE33BE01E106BF01E00CBF3B
:1000980000E00FBD0AE00EBD04E00BBD01EE0ABD95
:1000A80000E609BF00E205BF00E808B97894889522
:1000B800FECF0CE002BB38BA189540D3DA9451F45D
:1000C80004E0D02E8ED158D106D0FA9419F404E663
:1000D800F02E3BD0189501E0E01600E010E041F466
:1000E800F6FC06C0F3FC04C002E113E08D9A01C0DF
:1000F8008D9800BF13BFE4E8F0E0EC0DF31D099400
:1001080006C005C009C00DC011C015C019C004E063
:1001180009BD02EE08BD18C002E009BD01E708BD2F
:1001280013C001E009BD08E308BD0EC000E009BD29
:100138000CE908BD09C000E009BD0EE408BD04C013
:1001480000E009BD02E208BD089563956A30E0F059
:1001580060E073957630C0F070E083958A3098F04F
:1001680080E09395963078F090E0A395AED0AA30D1
:1001780010F0A0E0B395A43030F0B23020F0A0E049
:10018800B0E003D04FD0D6D0089500916200039517
:10019800009362000A3038F03092620000916300E8
:1001A80003950093630049D000916300011730F173
:1001B80044D010916200101708F101E0009362002A
:1001C80030926300009164000395009364000A3044
:1001D80038F0309264000091650003950093650043
:1001E80000916500013050F000916400033030F058
:1001F80001E0009364003092650001D008950091F9
:1002080068000395009368000A3058F0309268003F
:10021800009169000395009369000A3010F030924C
:100228006900089500916A00039500936A000830F8
:1002380018F001E000936A0008950091640010919D
:100248006500103009F00D5FEDE2F1E0E00FF31DFD
:10025800099409C008C00AC012C014C016C018C04A
:100268001AC01CC01EC013E002E008951DD0103053
:1002780019F412E009E0089513E000E0089513E08E
:1002880002E0089513E001E0089513E002E0089504
:1002980013E001E0089513E002E0089513E002E09E
:1002A800089513E001E00895109169000091680035
:1002B8001170113009F40E5F11E0003029F004309C
:1002C80019F0083009F010E0089500916600003038
:1002D80071F100916300003051F1013041F10330B8
:1002E80021F000916200053010F100916A0007309A
:1002F800F1F400916400033029F0009164000030AB
:1003080041F015C0A23099F4B03089F4A3E0B0E010
:10031800089500916700013051F0A33041F4B030E6
:1003280031F4A2E0B0E001E0009367000895309254
:1003380067000895009170000030E9F0013031F055
:10034800033021F000916A000630A8F400916C0097
:10035800081700916D00090700916E000A070091C7
:100368006F000B0741F401E0E02E009170000130AE
:1003780011F430927000089500916100003019F076
:100388000A95009361001091600000B30C7000930F
:100398006000101761F010916100103041F403FF04
:1003A80003C002FF03C003C0FFD001C0BDD112E0EB
:1003B80002FF1093610003FF1093610010916B001E
:1003C80002FF139510936B0010916100103019F41F
:1003D80010E010936B0010916B00143609F4ACD147
:1003E8000895CC27EBEFF1E0ED0FF31D099410C051
:1003F8000FC012C023C045C054C058C05CC062C002
:100408006BC07DC08EC09FC0ABC0B2C0B7C0BCC0FF
:100418009C01AD01C3E0089560FF0CC02091640009
:100428003091650030FF3AE04091620050916300DE
:10043800C6E008959C01AD01C3E008956030A1F0C5
:10044800653091F06330C9F06430B9F06830A8F4D1
:10045800209164003091650030FF3AE040916200DD
:1004680050916300C6E0089520916A0030916A00B7
:10047800206830684AE05AE008959C01AD01C3E065
:1004880008952AE030917000323021F0333019F4A9
:1004980037E001C035E0F4FC3AE04CE05BE0C2E054
:1004A800089579D0F4FC2AE0C3E0089574D0F4FCF0
:1004B8003AE0C3E008956FD0F4FC4AE0F4FC5AE057
:1004C800C3E008955BE04DE0F4FE30916600F4FC73
:1004D8003AE02AE0C2E00895F4FE52E0F4FC5AE063
:1004E800F4FE40E0F4FC4AE0F4FE30916900F4FCCC
:1004F8003AE0F4FE20916800F4FC2AE00895409167
:10050800620050916300F4FE20916400F4FE309183
:100518006500F4FC2AE0F4FC3AE030FF3AE0C6E07B
:100528000895209164003091650030FF3AE0F4FEB0
:1005380040916200F4FE50916300F4FC4AE0F4FC40
:100548005AE0C6E008955AE04AE020916A003091E6
:100558006A0020683068F4FC2AE0F4FC3AE0089568
:100568009B01F4FE2AE0F4FE3AE0AC01C3E00895F2
:100578009C01F4FC2AE0AD01C3E008959C01F4FC61
:100588003AE0AD01C3E008959C014AE05AE0F4FE68
:10059800AD01C3E0089520916C0030916D00409149
:1005A8006E0050916F000895E31411F0EE24089541
:1005B800E1EEF2E0ED0FF31D099410C00FC00EC07C
:1005C8000DC011C019C022C02BC03FC047C048C0D1
:1005D80063C080C088C08FC094C099C0CA9411F409
:1005E80006E0C02E0895009170000395043008F0CD
:1005F800002700937000089500916C0003950A305D
:1006080008F0002700936C0095DE089500916D00B6
:100618000395063008F0002700936D008BDE0895DF
:1006280000916E0010916F0003950A3010F00027BA
:100638001395123020F0043010F000271127009392
:100648006E0010936F0076DE0895009166000395A2
:10065800023008F000E0009366000895D0DD0895A8
:10066800009164000395009364000A3038F03092DA
:100678006400009165000395009365000091650092
:10068800013048F000916400033028F001E0009345
:10069800640030926500089500916200039500930C
:1006A80062000A3038F030926200009163000395CE
:1006B80000936300C2DD00916300011750F0BDDDB7
:1006C80010916200101728F001E000936200309248
:1006D8006300089500916A000395083008F001E06E
:1006E80000936A0008950EE3F02A60E0739576306F
:1006F80008F070E0089583958A3008F080E01ADEEB
:1007080008959395963008F090E014DE0895A39527
:10071800AA3010F0A0E0B395A43020F0B23010F069
:10072800A0E0B0E007DE08950E2DEE24003019F4A5
:10073800DA9509F4D7E00895D0E1089533240CE060
:1007480002BB0D2D023071F00330B1F00430D9F046
:10075800022F27FF2CD027FD2FD0C2FD0F7708BB13
:10076800909A0895032F37FF22D037FD2BD0C0FD74
:100778000F7708BB919A0895042F19D0C1FD0F7700
:1007880008BB949A0895052F003009F40AE00FD0A9
:1007980010917000103009F00F77D53028F0D8305C
:1007A80018F40068F4FE0F7708BB969A08950E3087
:1007B80090F4F7E0E2EE0BC00058083060F4F7E080
:1007C800E0EF05C00058083030F4F7E0E8EFE00F3C
:1007D800F31D049108950EEF0895C0F9A4B09992FD
:1007E80082F88090FF88C7E3FFA387878788A3865E
:0807F800FF8CC192C68C92AB8C
:00000001FF
